:020000040000FA
:0400000077EF00F0A6
:020004000000FA
:040008000FEF00F006
:040018000FEF00F0F6
:04001C001000106E52
:10002000D838116EA1B204D0F2B409D06AEF00F052
:10003000548E1138D86E103A1038A192100055BE67
:1000400049D054A604D000D08B6A8A6A03D08A684B
:100050008B6800D0222A090E226203D0010E226E84
:1000600000D02250E84E0ED0E84E11D0E84E14D009
:10007000E84E17D0E84E1AD0E84E1DD0E84E20D0FA
:10008000E84E23D08B704CC08AFF6AEF00F08B7271
:100090004DC08AFF6AEF00F08B744EC08AFF6AEF92
:1000A00000F08B764FC08AFF6AEF00F08B7E50C065
:1000B0008AFF6AEF00F08B7C51C08AFF6AEF00F084
:1000C0008B7A52C08AFF6AEF00F08B7853C08AFFA8
:1000D0006AEF00F0000ED76EFA0ED66E1138D86EA9
:1000E000103A1038F294A192B180F28E100099EC7F
:1000F00002F0496AF29E928E928C9484546A84B67D
:10010000548080BE548480BC548280AA54868B82E2
:100110006AEC08F082A407D08B926AEC08F082B4F3
:1001200002D0558E01D0559E55AE2BD000D0F29AFC
:10013000F294929E929CE8EC0AF078EC08F093EC32
:100140000AF067EC08F067EC08F067EC08F076EC72
:100150000BF0DEEC09F067EC08F067EC08F067ECF8
:1001600008F076EC0BF039EC0AF067EC08F067EC7D
:1001700008F067EC08F076EC0BF02BEC09F02FEFB1
:1001800001F099EC02F055BEF29A4C6A4D6A4E6A43
:100190004F6A506A516A526A536A00D0750E4D6EAA
:1001A0007D0E4E6E8C0E506E010E84EC02F0516E80
:1001B000040E84EC02F0526E000E84EC02F0536EDA
:1001C0004D824E82518254B608D04C1E4D1E4E1E9A
:1001D0004F1E501E511E521E531E67EC08F067EC56
:1001E00008F067EC08F04C6A4D6A4E6A4F6A506A34
:1001F000516A526A536A00D0020E84EC02F04C6ECF
:10020000000E84EC02F04D6E010E84EC02F04E6E96
:10021000010E84EC02F04F6E000E84EC02F0506E82
:10022000030E84EC02F0516E010E84EC02F0526E6B
:10023000050E84EC02F0536E4F825182538254B605
:1002400008D04C1E4D1E4E1E4F1E501E511E521EDB
:10025000531E67EC08F067EC08F067EC08F054A454
:1002600001D003D0080E3E6E03D0040E3E6E00D0C7
:1002700054A201D003D0040E3D6E03D0020E3D6E99
:1002800000D0F28E010EC26E50EC05F05CC019F089
:100290005BC018F00F0E5C6401D014D05C6204D017
:1002A000A00E5B6401D00ED0010E5C6001D016D0B0
:1002B0005C6401D035D0680E5B6001D00FD05B6408
:1002C0000DD02ED0899C548A568654A401D003D0D8
:1002D000080E3E6E27D0040E3E6E24D054A00DD0E2
:1002E000898C54A203D0080E3E6E02D0020E3E6EE0
:1002F00054AA0CD0549A568615D0569654A403D0BE
:10030000040E3E6E0FD0080E3E6E0CD0549A5696D8
:1003100054A403D0080E3E6E05D0020E3E6E02D0ED
:10032000569600D0050EC26E50EC05F05CC017F07A
:100330005BC016F00F0E5C6401D014D05C6204D078
:10034000A00E5B6401D00ED0010E5C6001D016D00F
:100350005C6401D035D0680E5B6001D00FD05B6467
:100360000DD02ED0899E548C568454A201D003D037
:10037000040E3D6E27D0080E3D6E24D054A00DD043
:10038000898E54A203D0040E3D6E02D0080E3D6E3D
:1003900054AC0CD0549C568415D0569454A203D01F
:1003A000020E3D6E0FD0040E3D6E0CD0549C569440
:1003B00054A203D0040E3D6E05D0080E3D6E02D04F
:1003C000569400D055AE04D080A802D03FEC03F084
:1003D00017C012F016C013F006EC06F01EC02BF08A
:1003E0001FC02CF020C02DF021C02EF019C012F03B
:1003F00018C013F006EC06F01EC02FF01FC030F03E
:1004000020C031F021C032F085EC06F01BC012F0A4
:100410001AC013F006EC06F01EC033F01FC034F013
:1004200020C035F021C036F043EC07F055AE07D0C0
:100430007CEC04F0DEEC04F080A85CD060D080A8F6
:1004400001D02BD02BC023F02CC024F02DC025F0E0
:100450002EC026F03DC03BF02FC027F030C028F062
:1004600031C029F032C02AF03EC03CF0F29EB3EC1D
:1004700002F0F28E56A407D0010E54A6E81E4C6E70
:100480004D6E4E6E4F6E56A6FCD6010E54A6E81E5B
:10049000506E516E526E536EF4D633C023F034C09A
:1004A00024F035C025F036C026F03FC03BF037C001
:1004B00027F038C028F039C029F03AC02AF040C0EF
:1004C0003CF0F29EB3EC02F0F28E56A807D0010E7B
:1004D00054A6E81E4C6E4D6E4E6E4F6E56BA02D04C
:1004E00056A2CFD6010E54A6E81E506E516E526E23
:1004F000536EC7D6A2EC03F000EC04F0C2D63FEC7A
:1005000003F0BFD682EF02F0E86601D0FC0CE84EA3
:10051000180CE84EB50CE84EB90CE84E590CE84EF4
:10052000E90CE84EED0CE84E380CE84EFD0CE84EB8
:10053000F90C000E936E946E3F0E926E8A6A8B6A6F
:10054000899E899C010EC26E3B0EC16E8C0EC06EE0
:10055000D40ED56E950EB16EF26AA06AF28EF28A52
:10056000F28CA0821200236606D03BB604D04C6AFF
:1005700054A64C1E09D0235084EC02F03BB6E8820E
:1005800054A6E81E4C6E00D024660AD03BB608D0B4
:100590003BB406D0236604D04D6A54A64D1E09D044
:1005A000245084EC02F03BB4E88254A6E81E4D6E61
:1005B00000D025660ED03BB60CD03BB40AD03BB27F
:1005C00008D0236606D0246604D04D6A54A64D1E7A
:1005D00009D0255084EC02F03BB2E88254A6E81E14
:1005E0004E6E00D0265084EC02F054A6E81E4F6EEA
:1005F00000D0276606D03CB604D0506A54A6501EE0
:1006000009D0275084EC02F03CB6E88254A6E81EDC
:10061000506E00D028660AD03CB608D03CB406D054
:10062000276604D0516A54A6511E09D0285084EC84
:1006300002F03CB4E88254A6E81E516E00D0296650
:100640000ED03CB60CD03CB40AD03CB208D02766E1
:1006500006D0286604D0526A54A6521E09D02950EA
:1006600084EC02F03CB2E88254A6E81E526E00D040
:100670002A5084EC02F054A6E81E536E120056A6CF
:1006800034D0400E3EEC0BF0050E14EC0BF0050ED2
:1006900014EC0BF0050E14EC0BF0050E14EC0BF043
:1006A000050E14EC0BF0050E14EC0BF0050E14EC1B
:1006B0000BF0050E14EC0BF0050E14EC0BF0050E10
:1006C00014EC0BF0050E14EC0BF0050E14EC0BF013
:1006D000050E14EC0BF0050E14EC0BF0050E14ECEB
:1006E0000BF0050E14EC0BF01200400E3EEC0BF07C
:1006F000436A19C042F018C041F0100E446EFA0E61
:10070000415CD8B001D006D0416E050E14EC0BF060
:100710004406F5D74206D8B0F7D700D0426A320E69
:10072000415ED8B001D002D0432AF8D7435014EC30
:100730000BF04406446601D01200200E14EC0BF0BE
:10074000F8D71200000E3F6204D0410E3EEC0BF0D1
:1007500004D0400E3EEC0BF000D0336606D03FB61E
:1007600004D0200E14EC0BF004D0300E332414EC23
:100770000BF03FA604D02E0E14EC0BF000D0346624
:100780000AD03FB608D03FB406D0336604D0200E5E
:1007900014EC0BF004D0300E342414EC0BF03FA416
:1007A00004D02E0E14EC0BF000D035660ED03FB600
:1007B0000CD03FB40AD03FB208D0336606D03466BE
:1007C00004D0200E14EC0BF004D0300E352414ECC1
:1007D0000BF03FA204D02E0E14EC0BF000D0300E24
:1007E000362414EC0BF0570E14EC0BF0200E14EC26
:1007F0000BF0200E14EC0BF0200E14EC0BF012009A
:1008000056AA19D0490E3EEC0BF0200E14EC0BF05A
:100810002D0E14EC0BF02D0E14EC0BF02D0E14EC31
:100820000BF02D0E14EC0BF06B0E14EC0BF0F40E21
:1008300014EC0BF01200000E406204D04A0E3EECA5
:100840000BF004D0490E3EEC0BF000D0376606D01A
:1008500040B604D0200E14EC0BF004D0300E372438
:1008600014EC0BF040A604D02E0E14EC0BF000D0CC
:1008700038660AD040B608D040B406D0376604D0F7
:10088000200E14EC0BF004D0300E382414EC0BF0D6
:1008900040A404D02E0E14EC0BF000D039660ED01C
:1008A00040B60CD040B40AD040B208D0376606D06B
:1008B000386604D0200E14EC0BF004D0300E39242E
:1008C00014EC0BF040A204D02E0E14EC0BF000D070
:1008D000300E3A2414EC0BF056A207D06B0E14EC39
:1008E0000BF0F40E14EC0BF01200F40E14EC0BF001
:1008F000200E14EC0BF01200000E3EEC0BF056A490
:1009000013D0200E14EC0BF02D0E14EC0BF02D0E6A
:1009100014EC0BF02D0E14EC0BF02D0E14EC0BF070
:10092000560E14EC0BF012002B6606D03DB604D028
:10093000200E14EC0BF004D0300E2B2414EC0BF032
:100940003DA604D02E0E14EC0BF000D02C660AD07D
:100950003DB608D03DB406D02B6604D0200E14EC72
:100960000BF004D0300E2C2414EC0BF03DA404D07A
:100970002E0E14EC0BF000D02D660ED03DB60CD030
:100980003DB40AD03DB208D02B6606D02C6604D008
:10099000200E14EC0BF004D0300E2D2414EC0BF0D0
:1009A0003DA204D02E0E14EC0BF000D0300E2E24FD
:1009B00014EC0BF0560E14EC0BF01200090E3EEC8A
:1009C0000BF056A616D0200E14EC0BF02D0E14ECE6
:1009D0000BF02D0E14EC0BF02D0E14EC0BF02D0E75
:1009E00014EC0BF0410E14EC0BF0200E14EC0BF099
:1009F00012002F6606D03EB604D0200E14EC0BF089
:100A000004D0300E2F2414EC0BF03EA604D02E0E92
:100A100014EC0BF000D030660AD03EB608D03EB4DD
:100A200006D02F6604D0200E14EC0BF004D0300E4C
:100A3000302414EC0BF03EA404D02E0E14EC0BF07A
:100A400000D031660ED03EB60CD03EB40AD03EB2D5
:100A500008D02F6606D0306604D0200E14EC0BF0C0
:100A600004D0300E312414EC0BF03EA204D02E0E34
:100A700014EC0BF000D0300E322414EC0BF0020E0C
:100A80003E6207D06D0E14EC0BF0410E14EC0BF02F
:100A90001200410E14EC0BF0200E14EC0BF01200BF
:100AA000500E576E01EE00F0C2804DEC08F0C2828D
:100AB000C2B258EF05F0C3CFEEFFC4CFEEFF572E02
:100AC000F6D7586A01EE01F011EE03F0EF50E7643B
:100AD00001D01BD0E76209D0ED52E552EF50E76438
:100AE00001D018D0E652EE5200D0E652E652010E86
:100AF000E2622CD0A10EE162E9D700D0ED6AEE6A85
:100B0000582A080E5862DED70CD0E1CFE9FFE2CFB9
:100B1000EAFFEBD7E1CFE9FFE2CFEAFFEE52E65280
:100B2000E4D7586A01EE01F011EE03F0EF660ED043
:100B3000ED52EE660BD0EE52EE52E652E652010E48
:100B4000EA62F4D79F0EE962F1D70ED0E76613D0C0
:100B5000E552E66610D0E652E652010EE262F6D7A2
:100B6000A10EE162F3D700D0ED6AEE6A582A080EB2
:100B70005862D8D71BD0EF50E76001D00BD0E762A6
:100B8000EAD7ED52E552EF50E76001D008D0E652C7
:100B9000EE52E1D7E1CFE9FFE2CFEAFFDCD7E1CFC8
:100BA000E9FFE2CFEAFFEE52E652D5D75B6A5C6A14
:100BB0005D6A500E586E01EE00F0EE505B26EE506E
:100BC0005C22D8A001D05D2A58065866F6D7200EC0
:100BD0005B26000E5C22000E5D22D8905D325C32F6
:100BE0005B32D8905D325C325B32D8905D325C32E1
:100BF0005B32D8905D325C325B32D8905D325C32D1
:100C00005B32D8905D325C325B3212001E6A1F6A22
:100C1000206A216A030E125CE80ED8B4135CD8A0D7
:100C200024EF06F0030E125CD8A024EF06F01BEFB1
:100C300006F024EF06F0126EE80E135C136ED8A0D7
:100C400012061E2A0AEF06F0640E135CD8B02FEFCE
:100C500006F012662DEF06F033EF06F01206136E63
:100C60001F2A24EF06F00A0E135CD8A03EEF06F010
:100C7000202A136E33EF06F013C021F013C021F0C9
:100C800012006F6A706A716A726A6D506B02F3CFFC
:100C90006FF0F4CF70F06E506C02F3CF71F0F4CFC0
:100CA00072F06D506C02F3507026F4507122E86AB5
:100CB00072226E506B02F3507026F4507122E86A73
:100CC00072221200200E676E626A616AD8906336E3
:100CD00064366536663661366236D8B07AEF06F02D
:100CE0006050625CD8A477EF06F05F50615CD8A0DA
:100CF00081EF06F05F50615ED8A062066050625ED0
:100D00006380672E66EF06F0120017C06CF016C005
:100D10006BF019C06EF018C06DF041EC06F07F0E5C
:100D2000676E960E686E980E696E000E6A6E6F5052
:100D3000675C705068587150695872506A5801E287
:100D400007D0080E3D6251D0020E3E624ED000D058
:100D5000880E6F26130E7022000E7122000E722272
:100D6000100E5F6E270E606E6FC063F070C064F08F
:100D700071C065F072C066F062EC06F064C01BF0F2
:100D800063C01AF0080E3D620FD0020E3E6203D01F
:100D9000080E3F6E77D0080E3E6203D0040E3F6E01
:100DA00071D0020E3F6E6ED0040E3D620FD0020E67
:100DB0003E6203D0040E3F6E65D0080E3E6203D043
:100DC000020E3F6E5FD0020E3F6E5CD0020E3E629E
:100DD00003D0020E3F6E56D0080E3E6203D0020EC4
:100DE0003F6E50D0000E3F6E4DD0F40E6F26010EB8
:100DF0007022000E7122000E7222E80E5F6E030E4A
:100E0000606E6FC063F070C064F071C065F072C056
:100E100066F062EC06F064C01BF063C01AF0080EC6
:100E20003D620FD0020E3E6203D0080E3F6E2AD004
:100E3000080E3E6203D0080E3F6E24D0040E3F6EB3
:100E400021D0040E3D620FD0020E3E6203D0080E88
:100E50003F6E18D0080E3E6203D0040E3F6E12D0D3
:100E6000020E3F6E0FD0020E3E6203D0040E3F6EA4
:100E700009D0080E3E6203D0020E3F6E03D0000E72
:100E80003F6E00D01200196604D0186602D0568A50
:100E90001200569A5692100E406E080E3D6204D013
:100EA0004046404640460BD0040E3D6203D04046CB
:100EB000404605D0020E3D6202D0404600D0080EEA
:100EC0003E6204D04042404240420ED0040E3E6298
:100ED00003D04042404208D0020E3E62FDD740425D
:100EE00040424042404200D017C06CF016C06BF048
:100EF000270E6E6E100E6D6E41EC06F0800E406295
:100F000001D00CD0400E406201D023D0200E4062B0
:100F100001D039D0100E406267D04ED0270E606EDF
:100F2000100E5F6E6FC063F070C064F071C065F04A
:100F300072C066F062EC06F063C06FF064C070F0DF
:100F400065C071F066C072F040424042404240428B
:100F50004BD0030E606EE80E5F6E6FC063F070C022
:100F600064F071C065F072C066F062EC06F063C0B8
:100F70006FF064C070F065C071F066C072F04042FE
:100F80004042404231D0000E606E640E5F6E6FC012
:100F900063F070C064F071C065F072C066F062EC1E
:100FA00006F063C06FF064C070F065C071F066C099
:100FB00072F04042404218D0000E606E0A0E5F6E22
:100FC0006FC063F070C064F071C065F072C066F00D
:100FD00062EC06F063C06FF064C070F065C071F041
:100FE00066C072F0404200D019C060F018C05FF0D7
:100FF0006FC063F070C064F071C065F072C066F0DD
:1010000062EC06F065C007F064C006F063C005F04E
:10101000D3EC0BF00F6601D00BD00FC037F00EC031
:1010200038F00DC039F00CC03AF04042568234D04E
:101030000E6601D00AD00EC037F00DC038F00CC0DB
:1010400039F00BC03AF0568227D00D6601D00CD093
:101050000DC037F00CC038F00BC039F00AC03AF0C0
:1010600040424042569218D00C6601D00BD00CC0C2
:1010700037F00BC038F00AC039F009C03AF04042EE
:1010800056920AD00BC037F00AC038F009C039F0C8
:1010900008C03AF0569200D01200190EE82E4EEF1A
:1010A00008F0120067EC08F067EC08F067EC08F055
:1010B00067EC08F067EC08F067EC08F067EC08F004
:1010C00067EC08F067EC08F067EC08F01200640EBB
:1010D0006EEF08F00A0E6EEF08F0010E466EF80E85
:1010E000456E452E71EF08F0462E6FEF08F01200A6
:1010F00076EC0BF0400E5BEC0BF0020E14EC0BF0F8
:10110000040E14EC0BF00E0E14EC0BF0010E14ECAC
:101110000BF00F0E14EC0BF0110E14EC0BF00F0E85
:1011200014EC0BF0000E14EC0BF0020E14EC0BF0B0
:10113000040E14EC0BF00E0E14EC0BF0110E14EC6C
:101140000BF01F0E14EC0BF0100E14EC0BF00E0E47
:1011500014EC0BF0000E14EC0BF0020E14EC0BF080
:10116000040E14EC0BF0000E14EC0BF00C0E14EC4F
:101170000BF0040E14EC0BF0040E14EC0BF00E0E3E
:1011800014EC0BF0000E14EC0BF0050E14EC0BF04D
:101190000A0E14EC0BF0000E14EC0BF00E0E14EC17
:1011A0000BF0110E14EC0BF0110E14EC0BF00E0EF4
:1011B00014EC0BF0000E14EC0BF00A0E14EC0BF018
:1011C000000E14EC0BF0110E14EC0BF0110E14ECDD
:1011D0000BF0110E14EC0BF0110E14EC0BF00E0EC4
:1011E00014EC0BF0000E14EC0BF0020E14EC0BF0F0
:1011F000040E14EC0BF0000E14EC0BF00E0E14ECBD
:101200000BF0110E14EC0BF0110E14EC0BF00E0E93
:1012100014EC0BF0000E14EC0BF0020E14EC0BF0BF
:10122000040E14EC0BF00E0E14EC0BF0110E14EC7B
:101230000BF01F0E14EC0BF0110E14EC0BF0110E52
:1012400014EC0BF0000E14EC0BF0000E3EEC0BF067
:1012500076EC0BF0120076EC0BF0400E5BEC0BF032
:10126000000E14EC0BF0000E14EC0BF0000E14EC5E
:101270000BF0000E14EC0BF0000E14EC0BF0000E53
:1012800014EC0BF0000E14EC0BF0000E14EC0BF051
:10129000100E14EC0BF0100E14EC0BF0100E14ECFE
:1012A0000BF0100E14EC0BF0100E14EC0BF0100EF3
:1012B00014EC0BF0100E14EC0BF0100E14EC0BF001
:1012C000180E14EC0BF0180E14EC0BF0180E14ECB6
:1012D0000BF0180E14EC0BF0180E14EC0BF0180EAB
:1012E00014EC0BF0180E14EC0BF0180E14EC0BF0C1
:1012F0001C0E14EC0BF01C0E14EC0BF01C0E14EC7A
:101300000BF01C0E14EC0BF01C0E14EC0BF01C0E6E
:1013100014EC0BF01C0E14EC0BF01C0E14EC0BF088
:101320001E0E14EC0BF01E0E14EC0BF01E0E14EC43
:101330000BF01E0E14EC0BF01E0E14EC0BF01E0E38
:1013400014EC0BF01E0E14EC0BF01E0E14EC0BF054
:101350001F0E14EC0BF01F0E14EC0BF01F0E14EC10
:101360000BF01F0E14EC0BF01F0E14EC0BF01F0E05
:1013700014EC0BF01F0E14EC0BF01F0E14EC0BF022
:10138000020E14EC0BF0040E14EC0BF00E0E14EC29
:101390000BF0110E14EC0BF01F0E14EC0BF0110EF1
:1013A00014EC0BF0110E14EC0BF0000E14EC0BF01F
:1013B000000E3EEC0BF076EC0BF01200000E3EEC53
:1013C0000BF0500E14EC0BF0490E14EC0BF0430E26
:1013D00014EC0BF02D0E14EC0BF0650E14EC0BF06E
:1013E000730E14EC0BF0200E14EC0BF0700E14ECDA
:1013F0000BF0610E14EC0BF06E0E14EC0BF0650E9E
:1014000014EC0BF06C0E14EC0BF06D0E14EC0BF0F6
:10141000010E14EC0BF0720E14EC0BF0030E14EC36
:101420000BF0420E3EEC0BF0760E14EC0BF0650E5A
:1014300014EC0BF0720E14EC0BF07A0E14EC0BF0B3
:10144000690E14EC0BF0050E14EC0BF03A0E14ECD4
:101450000BF0010E300F14EC0BF02E0E14EC0BF011
:10146000040E300F14EC0BF0000E300F14EC0BF0E8
:101470001200010E3EEC0BF0700E14EC0BF0610E3E
:1014800014EC0BF02D0E14EC0BF0650E14EC0BF0BD
:101490006C0E14EC0BF0650E14EC0BF06B0E14ECF0
:1014A0000BF0740E14EC0BF0720E14EC0BF06F0ECC
:1014B00014EC0BF06E0E14EC0BF0690E14EC0BF048
:1014C0006B0E14EC0BF0610E14EC0BF0430E3EECC3
:1014D0000BF0020E300F14EC0BF0000E300F14EC7A
:1014E0000BF0010E300F14EC0BF0010E300F14EC6A
:1014F0000BF02E0E14EC0BF0000E300F14EC0BF072
:10150000030E300F14EC0BF02E0E14EC0BF0010E4A
:10151000300F14EC0BF0050E300F14EC0BF02E0E08
:1015200014EC0BF01200410E14EC0BF0640E14ECF2
:101530000BF06A0E14EC0BF06F0E14EC0BF06E0E49
:1015400014EC0BF0200E14EC0BF0610E14EC0BF00D
:101550007A0E14EC0BF0200E14EC0BF0490E14EC88
:101560000BF0730E14EC0BF0740E14EC0BF0650E14
:1015700014EC0BF06E0E14EC0BF02C0E14EC0BF0C4
:10158000420E3EEC0BF0730E14EC0BF07A0E14ECE2
:101590000BF0650E14EC0BF0620E14EC0BF0620E07
:1015A00014EC0BF0200E14EC0BF06A0E14EC0BF0A4
:1015B000EF0E14EC0BF0760E14EC0BF0030E14ECA3
:1015C0000BF0740E14EC0BF0210E14EC0BF0120067
:1015D0008B908A808A9467EC08F067EC08F067ECDF
:1015E00008F067EC08F067EC08F08A928A968B980E
:1015F0008B9A8B9C8B9E8A8E8A8C8A9A8A986DECA9
:1016000008F08A866DEC08F08A968B988B9A8B8C02
:101610008B8E8A8E8A8C8A9A8A986DEC08F08A86DC
:101620006DEC08F08A961200F2AE01D002D056900E
:1016300001D05680F29E8A968A948A828A988A9AE3
:101640008A9C8A9E8B9E8B9C8B9A8B98E8B08A880A
:10165000E8B28A8AE8B48A8CE8B68A8EE8B88B8EBB
:10166000E8BA8B8CE8BC8B8AE8BE8B888A864DEC06
:1016700008F08A9656A01200F28E12008A968A927C
:101680008A988A9A8A9C8A9E8B9E8B9C8B9A8B883E
:10169000E8B08A88E8B28A8AE8B48A8CE8B68A8E8A
:1016A000E8B88B8EE8BA8B8CE8BC8B8A8A864DECC6
:1016B00008F08A9612008A968A928A988A9A8A9C58
:1016C0008A9E8B9E8B9C8B8A8B98E8B08A88E8B226
:1016D0008A8AE8B48A8CE8B68A8EE8B88B8EE8BA33
:1016E0008B8C8A864DEC08F08A9612008A968A9234
:1016F0008A888A9A8A9C8A9E8B9E8B9C8B9A8B98CE
:101700008A864DEC08F08A966DEC08F06DEC08F0D6
:101710001200000E3EEC0BF0200E14EC0BF014EC5B
:101720000BF014EC0BF014EC0BF014EC0BF014ECCD
:101730000BF014EC0BF014EC0BF014EC0BF014ECBD
:101740000BF014EC0BF014EC0BF014EC0BF014ECAD
:101750000BF014EC0BF014EC0BF01200400E3EEC0E
:101760000BF0200E14EC0BF014EC0BF014EC0BF05F
:1017700014EC0BF014EC0BF014EC0BF014EC0BF07D
:1017800014EC0BF014EC0BF014EC0BF014EC0BF06D
:1017900014EC0BF014EC0BF014EC0BF014EC0BF05D
:1017A00014EC0BF0120030D8F36ED8900BD020EE72
:1017B00000F0330EDF26DFB6F00BDFBE0F0BDE5E70
:1017C000D9A4F7D705360636073600360136023675
:1017D0000336F32EECD703380F0B0F6E03500F0BAD
:1017E0000E6E02380F0B0D6E02500F0B0C6E01388F
:1017F0000F0B0B6E01500F0B0A6E00380F0B096EAA
:1018000000500F0B086E1200006A016A026A036A38
:06181000180C09EF0CF0BA
:020000040030CA
:0100010038C6
:01000200F904
:01000300FEFE
:010005007B7F
:01000600BB3E
:01000800FCFB
:01000900BF37
:01000A00FFF6
:01000B00FFF5
:01000C00FFF4
:01000D00FFF3
:00000001FF
